:10000000DF298313B800B901B90D003039028030FF
:1000100003193802031C1228B51B12282030B80718
:100020000318B90A00303902F03003193802031CF2
:100030001C2883173030B807380884000800803047
:10004000A100FE303B2101303B217530AB00303048
:100050005C29A101A117B700FE303B2137083B29DD
:10006000B001B101B201B301A7123D21031C080088
:10007000D33E0319A7162D3EC63E031835280A3E67
:10008000031C3528AE00AD01AC01AB010A30AA005B
:100090008D212E082A07B0002B08B1000301031898
:1000A0000130B1072C08B200030103180130B20778
:1000B0002D08B300030103180130B307A50303198A
:1000C0006A283D21031C0800C63E03186A280A3E20
:1000D00003184228A71E7728B009B109B209B3094D
:1000E000B00A0319B10A0319B20A0319B30A300896
:1000F0000314C529A501B000B101A01125080319F9
:10010000A0150530A4002730AF0010309320033035
:10011000AF00E8309320AF0164309320AF010A3084
:10012000932030089A28AE003108AB003008AA00AE
:1001300071212A08AA00A4030319A0112508031994
:10014000A42824020318AB282A08031DA011A01913
:10015000AB28303E3B290800B00024080319C5290C
:100160003118831730088400000883130319C52948
:100170003B21B00AA403AD28B50005110510831674
:1001800005110510F030860583123508A018E62801
:100190003E30AB0080305C213330B400FB201330A4
:1001A000AB0088305C21FB2064305B21FB20643095
:1001B0005B212230B400FB202830E5200C30E52004
:1001C0000630E520A0143508E6282014B400201CD1
:1001D000F4280510033C031CF928F9200530AB0076
:1001E000DC305C21031408002014FE3C03190829AC
:1001F0000514B40E201C20100515F03086053408B7
:100200000F3986040511B40E2018FB2832305B210B
:100210003508C529E830AA000330AB00AE018316CB
:10022000861683120000861A2429FF30AE07031CAD
:10023000AA07031CAB07031CC5292E0A9630031915
:10024000AE000000232912290030AB0033305C21BE
:100250000830AF0037210310861E0314AE0C640073
:100260003129AF0B2A29372103142E08C529003064
:10027000AB00CC305C29A11BBC284208063A03190C
:100280000A290314C21F08000008840A0800831703
:100290008001840AFF3E031D4829C529AF01AE0035
:1002A000FF30AE07031CAF07031CC5290330AB00AA
:1002B000E5305C215029AB01F73EAA00AB09031CD5
:1002C0006729FE306329AA0703186229AA070000DC
:1002D0000000AB0F61296C292A1C70296F29702935
:1002E0000800B101B0011030B4002B0DB00DB10DFC
:1002F0002E08B0022F08031C2F0FB1020318872904
:100300002E08B0072F0803182F0FB1070310AA0DEE
:10031000AB0DB40B75292A08C5292030B400BE01E5
:10032000BF01C001C10103102A1CA4293008BE0767
:1003300031080318310FBF0732080318320FC00706
:1003400033080318330FC107C10CC00CBF0CBE0C1F
:10035000AD0CAC0CAB0CAA0CB40B932908001030FC
:10036000B900AB01AA01B50CB40C031CBD292E08C1
:10037000AA072F0803182F0FAB07AB0CAA0CB10C60
:10038000B00CB90BB3293008C529831383120313AA
:1003900000000800B4002408B50025070120340837
:1003A0008000C529B4002308B500340823070120C4
:1003B0000008C5298400A5018030C2003028A001B2
:1003C00007309F000130AF00F4304F21203084000F
:1003D00060304821A0308400503048212030840013
:1003E000303047211F2064304E218030A100C030C2
:1003F00029202030BC20BC205630BC204B30BC20F3
:100400003730BC204B30BC205230BC204A30BC209E
:100410002030BC204730BC205030BC205330BC20A2
:100420002030BC204330BC206C30BC206F30BC205E
:100430006330BC206B30BC202030BC20BC20073097
:10044000AF00D0304F21012B8316CD0A44308312E8
:10045000A30083164D088312D2218316CF002C30BF
:100460004F028312031D352A3B2A2C3083164F027C
:100470008312031D242A08008316CD0A4D08A13ECD
:1004800084000008CF002C304F028312031D492A3C
:100490004F2A2C3083164F028312031D3C2A08007A
:1004A000043083164B0283120319682A0630831620
:1004B0004B0283120319682A093083164B028312F8
:1004C0000319682A0B3083164B028312031D742A0A
:1004D0001F3083164A028312031C722A8316CB0A2A
:1004E0000130CA008312AE2A023083164B028312F7
:1004F000031D982A1E3083164A0203010318013097
:100500008312C300033083164C058312A800A9018F
:100510002908280403198E2A03018F2A0130430574
:100520000319962A8316CB0A0130CA008312AE2A19
:10053000203083164A028312031CA22A8316CB0A98
:100540000130CA0083120D3083164B028312031C44
:10055000AD2A8316CC0A0130CB00831208001F207D
:100560008030A100C03029202030BC20BC20BC201D
:10057000BC204E30BC206F30BC202030BC20473027
:10058000BC205030BC205330BC202030BC20643014
:10059000BC206130BC207430BC206130BC202030D5
:1005A000BC20BC20BC20BC20BC208030A1009430EA
:1005B00029205330BC206530BC207230BC2069300B
:1005C000BC206130BC206C30BC202030BC206930A5
:1005D000BC206E30BC207030BC207530BC20743024
:1005E000BC202030BC206D30BC206930BC20733072
:1005F000BC20BC206930BC206E30BC206730BC20E1
:10060000012B2030840060304821A030840050301D
:100610004821203084003030472101308316CD003E
:1006200083120A21031CAF2A243C031D102B0A212C
:10063000031CAF2A473C031D102B0A21031CAF2AC1
:10064000503C031D102B0A21031CAF2A473C031DFD
:10065000102B0A21031CAF2A473C031D102B0A2133
:10066000031CAF2A413C031D102B0A21031CAF2A97
:100670002C3C031D102B2530A5002508031403195D
:10068000462B0A21031CAF2AA5033D2BA801031406
:100690000A21031CAF2A2808A13E84002E088000EE
:1006A000A80A28080E3C031D472B0A21031CAF2A69
:1006B000243C031D552B0A21031CAF2A473C031D74
:1006C000552B0A21031CAF2A503C031D552B0A2130
:1006D000031CAF2A523C031D552B0A21031CAF2AD1
:1006E0004D3C031D552B0A21031CAF2A433C031D1F
:1006F000552B0A21031CAF2A2C3C031D552BA801A6
:1007000003140A21031CAF2A2808A5004430A400C2
:100710002E08CA21A80A28083C3C031D802B24224D
:100720008316CD0A44308312A30083164D0883122A
:10073000D2218316CE0041304E028312031DA12B1D
:10074000CF2B1F208030A100C03029205730BC2083
:100750006130BC206930BC207430BC206930BC20C2
:100760006E30BC206730BC202030BC206630BC20FE
:100770006F30BC207230BC202030BC204730BC2001
:100780005030BC205330BC202030BC206C30BC200A
:100790006F30BC206330BC206B30BC20012B01309B
:1007A0008316CD00831224222422242224222422F0
:1007B00024228316C801CD0A44308312A300831675
:1007C0004D088312D2218316CE0083122E30831659
:1007D0004E0283120319FF2B83164808B73E84008C
:1007E0004E088000C80ACD0A44308312A300831645
:1007F0004D088312D2218316CE008312E52BB73029
:10080000DA218316C400831231088316C500450817
:100810008312B500831644088312B4000130AF0080
:10082000CF30AE00AF21BA003108BB003B08AB00AF
:100830003A08AA00AF01FA30AE0071218316C60053
:1008400083122B088316C700831224228316C80143
:10085000CD0A44308312A30083164D088312D2219F
:100860008316CE0083122C3083164E028312031996
:100870004C2C83164808B03E84004E088000C80AFD
:10088000CD0A44308312A30083164D088312D2216F
:100890008316CE008312322C8316CD0A4430831285
:1008A000A30083164D088312D2218316CE00D030C8
:1008B0004E078312BA00FF300318013EBB00B5019A
:1008C0003A08B400AF010A30AE00AF218316CA0067
:1008D000CD0A44308312A30083164D088312D2211F
:1008E0008316CE00D0304E078312BA00FF300318B3
:1008F000013EBB003A088316CA07CD0A4430831272
:10090000A30083164D088312D2218316CE00D03067
:100910004E078312BA00FF300318013EBB00B50139
:100920003A08B400AF010A30AE00AF218316CB0005
:10093000CD0A44308312A30083164D088312D221BE
:100940008316CE00D0304E078312BA00FF30031852
:10095000013EBB003A088316CB07CD0A4430831210
:10096000A30083164D088312D2218316CE00D03007
:100970004E078312BA00FF300318013EBB00B501D9
:100980003A08B400AF010A30AE00AF218316CC00A4
:10099000CD0A44308312A30083164D088312D2215E
:1009A0008316CE00D0304E078312BA00FF300318F2
:1009B000013EBB003A088316CC078312BB014408F2
:1009C000BA003030BA02031CBB033B08B5003A083A
:1009D000B400AF010A30AE00AF21BA003108BB004D
:1009E000BD014508BC003030BC02031CBD033A0801
:1009F0003C078316C90004304B028312031C0B2DE5
:100A00000B3083164B02831203180B2D0A3083160A
:100A1000C90783120E2D0B308316C90783121830B5
:100A2000831649028312031C192D18308316C9023C
:100A3000CA0A8312502201308316CD008312BB01F3
:100A4000831622088312BA003030BA02031CBB039B
:100A5000BD01831621088312BC003030BC02031C88
:100A6000BD033D08B5003C08B400AF010A30AE003C
:100A7000AF21BC003108BD003A083C078316C20014
:100A800083123C223C228316C801CD0A4D08A13EA8
:100A900084000008CE0083122E3083164E0283128B
:100AA0000319612D83164808BD3E84004E0880005E
:100AB000C80ACD0A4D08A13E84000008CE0083126A
:100AC0004B2D3C228316CD0A4D08A13E8400000820
:100AD000C30083121F208030A100803029203230D3
:100AE000BC203030BC200230A50083164C08831295
:100AF0007B202D30BC200230A50083164B088312CA
:100B00007B202D30BC200230A50083164A088312BA
:100B10007B202030BC208030A1008B302920023087
:100B2000A5008316490883127B203A30BC20803010
:100B3000A1008E3029204608BC204708BC203A304E
:100B4000BC204808BC204908BC208030A100C0302F
:100B50002920A501831647088312B1008316460891
:100B60008312B0007D206B30BC207030BC20683018
:100B7000BC202030BC208030A100C8302920831642
:100B8000420883127A207330BC206130BC2074305C
:100B9000BC207330BC208030A100CF30292004302D
:100BA000A400B101BD30AC20831643088312BC20E1
:100BB0008030A100943029205008BC205108BC206E
:100BC000DF30BC205208BC205308BC205408BC2095
:100BD0005508BC205608BC205A08BC202030BC2038
:100BE0005C08BC205D08BC205E08BC20DF30BC2057
:100BF0005F08BC206008BC206108BC206208BC20E3
:100C00006308BC206708BC208030A100D4302920B4
:100C10004330BC206F30BC207530BC207230BC200B
:100C20007330BC206530BC202030BC200730A400CD
:100C3000B101B030AC20DF30BC202030BC205430BB
:100C4000BC207230BC207530BC206530BC20012B2C
:02400E00223F4F
:00000001FF
